:100000000C94A1020C94D9020C94D9020C94D9023C
:100010000C94D9020C94D9020C94D9020C94D902F4
:100020000C94D9020C94D9020C94192D0C94EB2D3C
:100030000C940F280C94D9020C94D9020C94D90278
:100040000C94D9020C94D9020C94D9020C94D902C4
:100050000C94C9230C94B3280C94D9020C94D902A3
:100060000C94D9020C94D9020C94D9020C94D902A4
:100070000C94D9020C94D9020C94D9020C94D90294
:100080000C94D9020C94D9020C94D9020C94D90284
:100090000C94D9020C94D9020C94D9020C94D90274
:1000A0000C94D9020C94D9020C94D902C405C4054D
:1000B000F005F005580683078307830776060F07C8
:1000C00020072007421D2D1D4D1D521D571D5C1D73
:1000D000611D661D6B1D701D751D7A1D7F1D841DA4
:1000E000891D8E1D931D981D9D1DA21DA71DAC1D54
:1000F000B11DB61DBB1DC01DC51DCA1DCF1D3A1E9D
:100100001C1FDD22DF22E422E722EA22ED22F02278
:10011000582E7F2E772F7F2E772FCB2EEE2E772FF8
:10012000452F542F29003A003B003C003D003E0083
:100130003F00400041004200430035001E001F0008
:100140002000210022002300240025002600270093
:100150002B0014001A000800150017001C001800DE
:100160000C001200130039000400160007000900FB
:100170000A000B000D000E000F003300E1006400C8
:100180001D001B00060019000500110010003600BC
:100190003700E000E300E2002C00E6006500E70025
:1001A000E400500051004F00440045004600470065
:1001B0004800B300B200AE000151560057002D00B8
:1001C0002E002A0049004A004B00530054005500FD
:1001D000610058002F00300038004C004D004E00E8
:1001E0005F0060005E005B00630031003400E500EA
:1001F0003200280052005C005D0059005A00620085
:10020000005CC15CC35CC45CC55CC65CC75CCA5CAA
:10021000CB5CCC5CCD5C0100010001000100010061
:1002200001000100010001000100010001000100C6
:1002300001000100010001000100010001000100B6
:1002400001000100010001000100010001000100A6
:100250000100010001000100010001000100010096
:100260000100010001000100010001000100010086
:100270000100010001000100010001000100010076
:10028000BE000100010001000100010001000100A9
:1002900001000100010001000100AA00A900010005
:1002A0000100010001000100010001000100010046
:1002B0000100010001000100010001000100010036
:1002C0000100010001000100010001000100010026
:1002D000BD0001000100010001000100000000005C
:1002E0000000000000000001010203040506080AE6
:1002F0000C0F1114181C2024292E33393F464C535F
:100300005B626A7179818A929AA2AAB2B9C1C8CF96
:10031000D5DCE1E7EBF0F4F7FAFCFDFEFFFEFDFCB7
:10032000FAF7F4F0EBE7E1DCD5CFC8C1B9B2AAA285
:100330009A928A8179716A625B534C463F39332EB7
:100340002924201C1814110F0C0A080605040302A6
:100350000101000000000000000000000001010198
:100360000101010101010202020202020202020372
:100370000303030303030304040404040404050542
:100380000505050606060606070707070708080805
:1003900008090909090A0A0A0B0B0B0C0C0C0D0DB4
:1003A0000D0E0E0E0F0F0F1010111111121213134C
:1003B0001414151516161717181819191A1A1B1BC5
:1003C0001C1D1D1E1E1F2020212222232424252621
:1003D00026272829292A2B2C2D2D2E2F3031323259
:1003E000333435363738393A3B3C3D3E3F40414265
:1003F000434445464748494A4C4D4E4F505153544B
:10040000555658595A5B5D5E5F61626465666869FE
:100410006B6C6D6F7072737577787A7B7D7E80827E
:10042000838587888A8C8E8F91939596989A9C9EC7
:10043000A0A2A3A5A7A9ABADAFB1B3B5B7BABCBED7
:10044000C0C2C4C6C9CBCDCFD1D4D6D8DBDDDFE2A4
:10045000E4E7E9EBEEF0F3F5F8FAFDFF10034800EE
:100460006E006100680031003000380000000E03AB
:1004700048006E00610068004B0042000000040369
:10048000090409023B00020100A0FA09040000016E
:10049000030101000921110100012240000705812B
:1004A00003080001090401000103000000092111F3
:1004B0000100012232000705820320000112010021
:1004C0000200000008EDFE0000020001020001052C
:1004D000010980A101850319012AB700150126B77A
:1004E00000950175108100C0050C0901A10185046A
:1004F00019012AA002150126A0029501751081009C
:10050000C005010906A101050719E029E715002525
:10051000019508750181029501750881010507198A
:100520000029FF150026FF009506750881000508C3
:100530001901290595057501910295017503910130
:10054000C00011241FBECFEFDAE0DEBFCDBF04B67E
:1005500003FE18C08091E4049091E504A091E604A4
:10056000B091E7048730904BA740B04B59F41092FC
:10057000E4041092E5041092E6041092E704E0E02F
:10058000F8E3099512E0A0E0B1E0E2E1F2E602C092
:1005900005900D92A438B107D9F724E0A4E8B2E0A1
:1005A00001C01D92A43EB207E1F70E94C2130C9451
:1005B00007310C940000CF93811113C0C62F81E046
:1005C0000E94C708882331F0CC2311F08DEB07C0BF
:1005D0008EEB05C0CC2311F089EA01C08AEA0E94A3
:1005E000720581E0CF9108950E944D2781FF03C0DD
:1005F00020E04FEF0CC080FF04C020E040E06FEF30
:1006000007C082FF02C02FEF01C020E040E060E0A1
:100610008EE190E00C94671781E0089581E00895E1
:100620000C940E0308950C9412031F93CF93DF9341
:1006300000D000D01F92CDB7DEB749835A836B83B9
:100640003091870289819A81311114C0662359F053
:10065000222349F00E94DC09182F682F89819A8192
:100660000E94850903C00E94B009182F69817A8110
:10067000812F04C00E94DC0969817A810F900F905C
:100680000F900F900F90DF91CF911F910C942D112F
:10069000FC01262F408151816281738184810C94F9
:1006A000150381E00895CF93DF93EC0160E00E9491
:1006B0004803BE01DF91CF910C9413030C94731285
:1006C0000C946F1208950E940F080E9462032FEF8E
:1006D00084E39CE0215080409040E1F700C000009E
:1006E0000C94D9280F931F93CF93DF938C0161E073
:1006F0000E944803EC01B8010E941003882309F40A
:100700004BC0B801CE010E94CE22882309F444C018
:10071000B801CE010E94E5268823F1F1B801CE018F
:100720000E9490248823C1F1B801CE010E94412685
:10073000882391F1B801CE010E941721882361F12D
:10074000F8018281882309F1CB358DE5D807C1F006
:1007500050F4C115FCE5DF0781F0CF3DDC45A9F47D
:100760000E94130F19C0CC35EDE5DE0761F0CD35E1
:10077000DD4559F40E94560E08C00E9463030CC068
:100780000E945F0E02C00E94620EC801DF91CF91ED
:100790001F910F910C940C0380E0DF91CF911F917A
:1007A0000F9108950E94F12780E00E9486230E9405
:1007B0007C1C0E94F80381E00C9409200E94F22125
:1007C0000E94FB0380E00E9409200C94F727089503
:1007D0000C94E70381E008950C94EA030895CF9305
:1007E000C82F0E94E8038C2F0E94EC03CF9108953C
:1007F00080E00C94EF030E9441270C94EF030E94C9
:10080000412790918602891721F0809386020C94EB
:10081000EF030895CF93DF93CDB7DEB72B970FB6D5
:10082000F894DEBF0FBECDBF4F83588769877A87A4
:100830008B8761110E94A20D9E012F5F3F4F86E0C2
:10084000F90111928A95E9F785E0FE013796D90101
:1008500001900D928A95E1F789819A814C815D81A1
:10086000452B31F09F3F31F491E08F3F19F403C0E5
:1008700091E001C090E090FF09C049815A816B81ED
:100880007C818D819E810E94C30C05C0C9010E949C
:1008900051038111F2CF2B960FB6F894DEBF0FBE35
:1008A000CDBFDF91CF910895FC01808191810E949D
:1008B0001E0A0895CF93882309F49CC0C82F82385C
:1008C000C1F40E94412781FD95C069E38091D10167
:1008D0009091D2010E94C9270E94C40D2FEF81EE92
:1008E00094E0215080409040E1F700C0000069E3AF
:1008F00019C0833801F50E94412780FD7BC063E564
:100900008091D1019091D2010E94C9270E94C40D0B
:100910002FEF81EE94E0215080409040E1F700C03D
:10092000000063E58091D1019091D2010E94CB2714
:10093000CF910C94C40D8438C1F40E94412782FDEC
:1009400059C067E48091D1019091D2010E94C927DA
:100950000E94C40D2FEF81EE94E021508040904022
:10096000E1F700C0000067E4DDCF8CEF8C0F813A27
:10097000D0F46C2F8091D1019091D2010E949327E5
:10098000882349F06C2F8091D1019091D2010E946F
:10099000CB270E94C40D6C2F8091D1019091D20180
:1009A0000E94C927C5CF80E28C0F883048F4C770F9
:1009B00081E001C0880FCA95EAF70E94850DB8CF83
:1009C000EBE5EC0FE33040F4F0E0E55EFD4F8081B5
:1009D00090E0CF910C945B27C85AC73158F4EC2FA4
:1009E000F0E0EE0FFF1FE351FE4F80819181CF9128
:1009F0000C947127CF910895882309F45BC0682F68
:100A0000823879F40E94412781FF54C069E38091C4
:100A1000D1019091D2010E94C9270E94C40D69E3BF
:100A200010C08338B1F40E94412780FF43C063E5C2
:100A30008091D1019091D2010E94C9270E94C40DDA
:100A400063E58091D1019091D2010E94CB270C9453
:100A5000C40D843879F40E94412782FF2BC067E4DB
:100A60008091D1019091D2010E94C9270E94C40DAA
:100A700067E4E7CF8CEF860F813A18F380E2860FA8
:100A8000883048F4677081E001C0880F6A95EAF702
:100A90000E948B0DDCCF8BE5860F833020F480E045
:100AA00090E00C945B27685A673120F480E090E076
:100AB0000C94712708951F93CF93DF93182FEB01A8
:100AC0000E945A04209741F08FE99FE00197F1F7C7
:100AD00000C000002197F6CF812FDF91CF911F91A9
:100AE0000C94FC04893319F060E070E002C060E50A
:100AF00070E00C945B05882321F00E94850D0C9416
:100B0000C40D0895882321F00E948B0D0C94C40D10
:100B10000895CF92DF92EF92FF920F931F93CF939E
:100B2000DF937C01D62FC72FFC011281058102952E
:100B30000F700E947B0D8823B9F01123A9F08C2F30
:100B4000807F803421F080E28D0F883068F08091C2
:100B5000420482FD09C082E00E94240E0E947B0DA7
:100B600091E0D82ED92601C0D12CCC2EC2948FE092
:100B7000C8228C2D90E08C30910508F0C4C1FC0196
:100B8000EA5AFF4F0C9405308C2F807FCF7088235A
:100B900011F0C295C07F112399F0CC2309F49FC1B5
:100BA00080E28D0F883010F0D11104C08C2F0E948C
:100BB000850D03C08C2F0E94950D0E94C40D8FC11E
:100BC0008D2F0E94FC04CC2309F49DC180E28D0F7F
:100BD000883038F1DD2329F18C2F0E949B0D24C031
:100BE0008C2F807FCF70803211F0C295C07FDD23C3
:100BF00019F0D130A1F13DC08091420482FF17C0AD
:100C0000112349F0CC2329F08C2F0E94850D0E94DE
:100C1000C40D80E065C180E00E94FC04CC2309F48F
:100C200072C18C2F0E948B0D0E94C40D6CC11123C8
:100C300071F0002341F0013031F40E94A50D8C2B9E
:100C40000E94AD0D60C10E94A50D8C2B1DC000231C
:100C500019F0013009F457C10E94BA0D25C01123C3
:100C600021F0063008F04FC10EC0053008F04BC12E
:100C70001BC0112361F0002331F0F701858180FF53
:100C80002EC18F7085838C2F0E947B053CC1002371
:100C900059F0D93309F034C1FFEF07EE13E0F150FA
:100CA00000401040E1F72AC18C2F0E9482052BC121
:100CB0008C2F86958695837019F0813061F023C161
:100CC000112321F08D2F9C2F937002C080E090E0C3
:100CD0000E945B2720C1112321F08D2F9C2F937040
:100CE00002C080E090E00E94712715C18C2F8370B4
:100CF00009F047C011110BC12D2F229526952770A1
:100D0000220F220F6D2F6F70862F90E0A0E0B0E0D1
:100D1000022E04C0880F991FAA1FBB1F0A94D2F786
:100D2000D4FF10C04FE050E060E070E004C0440F1A
:100D3000551F661F771F2A95D2F7409550956095ED
:100D4000709503C040E050E0BA01C695C695C370E7
:100D50008A019B01082B192B2A2B3B2BC901B801B7
:100D6000C23049F058F4C13019F00E947B08CFC05E
:100D70000E946908CCC00E948D08C9C00E94670803
:100D8000C6C0112319F08C2F817001C0869588236D
:100D900009F4BDC02D2F229526952770220F220F12
:100DA0006D2F6F70862F90E0A0E0B0E0022E04C09F
:100DB000880F991FAA1FBB1F0A94D2F7D4FF10C037
:100DC0004FE050E060E070E004C0440F551F661F24
:100DD000771F2A95D2F7409550956095709503C07E
:100DE00040E050E0BA01C695C695C3708A019B01E8
:100DF000082B192B2A2B3B2BC901B801C23049F013
:100E000058F4C13019F00E94600981C00E944E0957
:100E10007EC00E9472097BC00E94A10878C0CF707A
:100E2000112339F08C2F0E94E7088D2F0E947B053B
:100E30006EC08D2F0E9482058C2F0E94080967C00A
:100E4000D23F21F128F4D03F41F0D13FC1F043C05F
:100E5000D33F19F1D43F79F03EC0112341F0053062
:100E600008F051C08C2F8F710E942D094CC00630A4
:100E700008F049C0F7CF8091420482FF18C01123C7
:100E800039F08C2F8F710E94E7083DC01123C9F300
:100E90008C2F8F710E94080936C0112329F08C2FE6
:100EA0008F710E94D2082FC00E94AD082CC0112360
:100EB00049F0CF718C2F0E94E70863E08C2F0E94CD
:100EC000090E21C081E00E94240E0230E0F082E091
:100ED0000E94240E18C0112331F0002391F28D2FAF
:100EE0000E945A0410C0002399F2D93349F41FEF2D
:100EF00027EE33E0115020403040E1F700C0000001
:100F00008D2F0E94FC0488EF8C0D843020F40E9409
:100F100041270E94EF03DD20C9F00E94770D80FD7C
:100F200015C0F70112820E94710D0E94E708C701E7
:100F30000E94C7070E94710DDF91CF911F910F9101
:100F4000FF90EF90DF90CF900C940809DF91CF9144
:100F50001F910F91FF90EF90DF90CF9008950F9326
:100F60001F93CF93DF93EC01688179818A810E947E
:100F7000290A8C010E9484090E945508B801CE01FB
:100F80000E948905DF91CF911F910F910895CF9312
:100F9000DF93EC01988189812B813C81232B31F0F7
:100FA0008F3F31F481E09F3F19F403C081E001C01D
:100FB00080E080FD1DC0CE010E947203811110C02F
:100FC0000E947B0D8823A1F08A81882389F080917B
:100FD000420482FD0DC082E0DF91CF910C94240E7B
:100FE000CE010E94AF07CE01DF91CF910C94530345
:100FF000DF91CF91089580E090E00E945B2780E030
:1010000090E00E9471270E94A20D0C94C40D809163
:10101000D1019091D2010E94CD270C94FB070E9430
:10102000920D0C94070892959F70963079F010F409
:10103000925001C09A50923068F4803F69F018F4E1
:10104000883E40F409C0843F29F406C0883E20F061
:10105000813F11F080E0089581E00895FC018081D6
:1010600091810E941E0A0E9413080895CF93DF9376
:1010700000D000D01F92CDB7DEB70F900F900F9029
:101080000F900F90DF91CF910895CF93DF9300D011
:1010900000D000D0CDB7DEB726960FB6F894DEBFED
:1010A0000FBECDBFDF91CF910895089508950C94A0
:1010B00056080C9457080E9459086093D202709306
:1010C000D3028093D4029093D5020C94FB070C9426
:1010D0005B080F931F930091D2021091D3022091CD
:1010E000D4023091D502602B712B822B932B1F9150
:1010F0000F910C945B080F931F930091D2021091F3
:10110000D3022091D4023091D5026023712382232F
:1011100093231F910F910C945B080F931F930091E1
:10112000D2021091D3022091D4023091D5026027CF
:101130007127822793271F910F910C945B080C94C1
:1011400056080E949F086093CE027093CF0280934E
:10115000D0029093D1020C94FB0760E070E0CB01C9
:101160000C94A108611571058105910529F481E0B0
:10117000442361F080E00895DC01CB0104C0B69502
:10118000A795979587954A95D2F781700895482F2E
:101190006091CE027091CF028091D0029091D102E5
:1011A0000C94B2080F931F9341E050E060E070E0B0
:1011B0008A019B0104C0000F111F221F331F8A9553
:1011C000D2F7C901B8011F910F910C94A1080F9398
:1011D0001F9341E050E060E070E004C0440F551FF1
:1011E000661F771F8A95D2F78091CE029091CF0229
:1011F000A091D002B091D1028A019B01082B192B3A
:101200002A2B3B2BC901B8011F910F910C94A10807
:101210000F931F9341E050E060E070E004C0440F82
:10122000551F661F771F8A95D2F740955095609598
:1012300070958091CE029091CF02A091D002B09192
:10124000D1028A019B01082319232A233B23C901C8
:10125000B8011F910F910C94A1080F931F9341E0C7
:1012600050E060E070E004C0440F551F661F771F18
:101270008A95D2F78091CE029091CF02A091D002B0
:10128000B091D1028A019B01082719272A273B2701
:10129000C901B8011F910F910C94A1080F931F93DE
:1012A0000091CE021091CF022091D0023091D10254
:1012B000602B712B822B932B1F910F910C94A10803
:1012C0000F931F930091CE021091CF022091D00274
:1012D0003091D10260237123822393231F910F91B8
:1012E0000C94A1080F931F930091CE021091CF028E
:1012F0002091D0023091D102602771278227932755
:101300001F910F910C94A10808952BE0929F800DDE
:101310001124E82FE695E695E695877051E001C027
:10132000550F8A95EAF785E0E89FF0011124E85708
:10133000FD4F20E030E070E04081CB01022E02C082
:10134000969587950A94E2F7817081958427852385
:10135000842781932F5F3F4F2530310569F708952A
:101360002BE0929F800D1124682F669566956695F7
:10137000982F977085E0689FB001112440E050E0FD
:1013800080E0FB01E40FF51FE857FD4F208130E0BE
:10139000092E02C0369527950A94E2F7217033276B
:1013A000042E01C0220F0A94EAF7822B4F5F5F4F91
:1013B0004530510531F70895BF92CF92DF92EF92F9
:1013C000FF920F931F93CF93DF938C01C090CE02B7
:1013D000D090CF02E090D002F090D1028091D20262
:1013E0009091D302A091D402B091D502C82AD92AF3
:1013F000EA2AFB2ACFE1D0E0D701C6010C2E04C0B7
:10140000B695A795979587950A94D2F780FD04C065
:10141000219790F7B12C07C0BC2EB8018C2F0E94E9
:1014200040110197A9F38B2DDF91CF911F910F915F
:10143000FF90EF90DF90CF90BF900895CF93DF9310
:10144000EC010E94DC09BE010E944011DF91CF91A6
:1014500008951F93CF93DF93EB0190918702992317
:1014600021F0CB010E941E0A13C0882349F0CB0152
:101470000E94DC09182F682FCE010E94850904C044
:10148000CB010E94B009182FBE01812F0E9440118C
:10149000DF91CF911F9108951F93CF93DF93C09158
:1014A000D60216E08091D702C81799F0D0E01C9FB1
:1014B000F0011D9FF00D1124E852FD4F4081518134
:1014C00062817381848195810E9445082196C7704D
:1014D000E9CFDF91CF911F9108954091080350917A
:1014E000090360910A0370910B0380910C039091A2
:1014F0000D030C944508EF92FF920F931F93CF9327
:10150000DF9380910D0382958F7009F065C0809103
:101510000A03882309F460C08091D602F090D702B4
:10152000109108030091090360910B0370910C0363
:1015300091E01F3F09F090E0C091CF01D091D00120
:10154000292F96E0E92E8F1509F446C06115710523
:1015500021F00F3F21F030E003C031E001C0322F15
:1015600090E030FD36C0E89EF001E99EF00D1124B8
:10157000DF01A852BD4F11963C911197301329C03D
:101580003C91311326C012963C911297311121C023
:1015900013964D915C911497461B570B4C175D07A2
:1015A000C0F480910D038F70806180930D03E3522E
:1015B000FD4F80818F708061808388E093E00E947E
:1015C000C707DF91CF911F910F91FF90EF900C947F
:1015D0004C0A01968770B7CFDF91CF911F910F9181
:1015E000FF90EF9008959F92AF92BF92CF92DF92BB
:1015F000EF92FF920F931F93CF93DF93CDB7DEB798
:1016000061970FB6F894DEBF0FBECDBF8C0185E0A9
:10161000F801DE011D9601900D928A95E1F7D8013F
:101620001296EC9090910803E091090320910B032E
:1016300030910C032115310531F0EF3F31F481E099
:101640009F3F19F403C081E001C080E0B82FB17062
:101650009B2E80FD47C1D8014C9111965C9111974A
:101660001396AD90BC90149788E0C82E83E0D82ED6
:10167000F0900A03B501621B730B2091CF013091EA
:10168000D001FF2009F4D9C080910D0362177307C0
:1016900008F095C0282F207F09F052C05E1313C0B8
:1016A000491311C0FE2CE1100EC08F708061809331
:1016B0000D030E946D0AC6010E94C70780910D03A9
:1016C000F80185834DC1AB2831F05F3F31F481E0F3
:1016D0004F3F19F403C081E001C080E080FD03C0EA
:1016E00081E08E2502C080E090E0F82FF170FF2E9F
:1016F00080FF1CC08091D6022091D70236E082176D
:1017000009F40BC190E0389FF001399FF00D1124CE
:10171000E852FD4F6181561306C06081461303C035
:101720006281E61203C001968770E9CFFE2CEE209D
:1017300009F416C180910D03816080930D0354C09C
:101740005E1306C0491304C0E11002C0F80199C03D
:10175000C8010E942E08882361F1EE2051F12091EA
:101760000D03822F82958F7090E0029774F0809124
:1017700008039091090398878F831986BB86AA86F0
:101780002C87CE0107960E94C70786E0F801A8E0E3
:10179000B3E001900D928A95E1F70E947B0A0E94C6
:1017A0006D0A0AC05E1711F1C8010E942E0881114E
:1017B0002CC0C8010E94C707FF24F394D1C0282F72
:1017C000207F81F77A2DB98AA88A6E2D89890E9497
:1017D000360888E093E00E94C70786E0D6011D9294
:1017E0008A95E9F70E946D0AF12CBAC04913DCCF43
:1017F000E110DACFF8018583C8010E94C70786E0AF
:10180000D6011D928A95E9F7ABC0EE2091F22091A6
:101810000D03822F82958F7090E002970CF4B5CF64
:1018200080910803909109039A8389831B82BD826A
:10183000AC822E83CE010196A6CF6217730708F003
:1018400044C0FE2CEE2009F4B4CF5E1330C049131F
:101850002EC020910D0320FD21C0822F82958F7014
:10186000482F50E041155105C9F0F80125834F304C
:10187000510541F08F5F982F9295907F822F8F7046
:10188000892B8583C8010E94C70786E0F801A8E07C
:10189000B3E001900D928A95E1F73CC086E0F80133
:1018A000A8E0B3E001900D928A95E1F759C0C80114
:1018B0000E942E08811169CF80910D038160809371
:1018C0000D03C8010E94C7074BC07A2DB98AA88AA8
:1018D0006E2D89890E94360886E0D6011D928A9570
:1018E000E9F718C0EE2009F464CFC8010E942E0861
:1018F000F82E882309F45DCF86E0F801A8E0B3E074
:1019000001900D928A95E1F788E093E00E945404DB
:101910000E947B0A0E946D0A23C04D875E878D85D9
:101920009E850E941E0A292F22952F70223028F4AE
:101930009F7039F0811105C00BC0243028F49F70CE
:1019400049F4805E883020F0C8010E94C7079F2CB0
:10195000F92C06C0D80115969C91907F91F7F8CF8D
:101960008F2D61960FB6F894DEBF0FBECDBFDF910D
:10197000CF911F910F91FF90EF90DF90CF90BF908C
:10198000AF909F9008951F93CF93DF93CDB7DEB7AD
:101990002C970FB6F894DEBF0FBECDBF4F8358878C
:1019A00069877A878B879C87CE0107960E94F30A06
:1019B0008823D1F09F8188852A853B85232B31F0B0
:1019C0008F3F31F481E09F3F19F403C081E001C0F3
:1019D00080E080FD47C04F81588569857A858B8579
:1019E0009C850E9445083EC086E0FE013796DE01D8
:1019F000119601900D928A95E1F7FF81E8856A853D
:101A00007B856115710531F0EF3F31F481E0FF3FD7
:101A100019F403C081E001C080E080FD23C0209163
:101A2000D70230E0C9010196877099274091D6020C
:101A300050E084179507F1F1F983EA837D836C8385
:101A400096E0929FD001939FB00D1124A852BD4FF4
:101A5000FE01319601900D929A95E1F78093D7029D
:101A60000E944C0A16E08091D6029091D702891705
:101A700071F1189FC001112488529D4F0E94F30AF2
:101A8000882329F1E091D6021E9FF0011124E8522B
:101A9000FD4F4081518162817381848195810E94D3
:101AA00045088091D60290E001968770992780932F
:101AB000D602D9CF0E940F081092D7021092D602F8
:101AC000E8E0F3E086E0DF011D928A95E9F72C96C5
:101AD0000FB6F894DEBF0FBECDBFDF91CF911F913F
:101AE0000895809116038595859585950895809133
:101AF00016038770089590911603977081E009F49A
:101B000080E0089580912103089590912103892B0D
:101B100080932103089580959091210389238093D8
:101B20002103089510922103089590912003892B99
:101B300080932003089580959091200389238093BA
:101B400020030895109220030895809117030895AB
:101B500008950C94A80D0C94A90D9091420492FD47
:101B600008C090911703981721F0809317030C94E5
:101B7000AB0D089580911703882329F01092170365
:101B800080E00C94AB0D0895CF93DF93E091D101E9
:101B9000F091D201809121038083E091D101F091F5
:101BA000D201908180912003892B8083809117033B
:101BB000882381F0E091D101F091D2019081892BAD
:101BC00080838091D1019091D2010E948727811159
:101BD0000E94BA0DC091D101D091D20148E050E0ED
:101BE0006EE073E0CE010E948130892B69F088E0BD
:101BF000FE01AEE0B3E001900D928A95E1F7CE01CF
:101C0000DF91CF910C945027DF91CF9108950C94E0
:101C1000A80D9091420492FD10C098E0899F900118
:101C20001124262B209316030E94E70880911603A7
:101C30008595859585950C94070E0C94E708109270
:101C4000160380E00C94070E2091160380958223E2
:101C500080931603982F977099F430E0482F082E40
:101C6000000C550B2417350759F09091420492FD52
:101C700007C08595859585950E9408090C941F0ECF
:101C800008959091420492FB222720F9281769F0C9
:101C900080FB92F990934204809141049091420418
:101CA0000E948F0E82E00C94240E089580914204CD
:101CB00082FB882780F991E089270C94410E81E00E
:101CC0000C94410E80E00C94410E6FEF7FEF80E0AA
:101CD00090E00C94DA3080E090E00E94A63021E0A1
:101CE000893E9E4F09F020E0822F089582E090E027
:101CF0000C949E3083E090E00C949E30CF9384E06F
:101D000090E00E949E30C82F82E290E00E949E30B8
:101D10002C2F30E0A901582BCA01CF910895CF9301
:101D2000C92F682F84E090E00E94BC306C2F82E2C3
:101D300090E0CF910C94BC30AB01BC018FE090E0FF
:101D40000C94CE30AB01BC0183E190E00C94CE301A
:101D500060E070E0CB010C94A20E60E070E0CB017B
:101D60000E949C0E0C94A80E69EE7EEF80E090E03D
:101D70000E94DA3060E082E090E00E94BC3060E0D7
:101D800083E090E00E94BC301092D2021092D30205
:101D90001092D4021092D50260E084E090E00E949C
:101DA000BC3060E082E290E00E94BC3060E085E000
:101DB00090E00E94BC3060E086E090E00E94BC3081
:101DC0006FEF87E090E00E94BC3040E050E0BA0145
:101DD00088E090E00E94CE3060E08DE090E00E94CC
:101DE000BC3040E050E0BA0188E190E00E94CE3083
:101DF00060E087E190E00E94BC3040E050E0BA0132
:101E00008CE190E00E94CE3060E070E080E290E0F3
:101E10000E94DA3040E050E0BA0188E190E00E9490
:101E2000CE300C94AD0E0C94B40E682F8EE090E082
:101E30000C94BC300E947C2860933E0370933F0357
:101E4000809340039093410360933A0370933B0364
:101E500080933C0390933D0308950E947C286093F7
:101E60003E0370933F03809340039093410360933C
:101E700036037093370380933803909339030895A2
:101E800085B7806885BF85B7806885BF089581E084
:101E900008950C94470F08950C944B0F0C944B0F1E
:101EA0000C944E0F0C944B0F0C94520F0C944B0F40
:101EB0000E94400F8CE192E10E9437270E94560F4A
:101EC0000C94540F0E944C0F0C944B0F0E9436122E
:101ED0000E94EE030E944F240C94EB1F0E9467287F
:101EE0000E941B130E94660F0E94F2210E94E125AE
:101EF0000C94500F5F926F927F928F929F92AF924D
:101F0000BF92CF92DF92EF92FF920F931F93CF93E6
:101F1000DF93CDB7DEB72A970FB6F894DEBF0FBEBA
:101F2000CDBF0E943013E82E81110E941A0F32E2B9
:101F3000832E33E0932E00E010E0502E802F0E947D
:101F40005A125C01F401619071904F016826792664
:101F500061147104B1F40F5F1F4F0A30110569F766
:101F60008FEF89838A831B820E9470288160782F7B
:101F70009D838C8349815A816B818D810E940A04E3
:101F800043C08091420381FD0E946312F12CCC2456
:101F9000C394D12CC3018C219D21892B71F10E9406
:101FA000490FAC20BD208823A1F0FE825F8281E032
:101FB000A114B10409F480E088870E947028816030
:101FC000782F9A8789874E815F8168858A850E94EC
:101FD0000A04000F111FF801EE5DFC4F8081918112
:101FE000C826D926D182C08241E0AB2809F440E05E
:101FF0006F2D852D0E94581C07C0F394CC0CDD1C5E
:10200000FBE0FF12C7CFA7CF81E0E11001C080E065
:102010002A960FB6F894DEBF0FBECDBFDF91CF91E9
:102020001F910F91FF90EF90DF90CF90BF90AF90F6
:102030009F908F907F906F905F9008950E947A0F8D
:102040000E947C1C0E94B3230E94F42581110E94EF
:102050002D0F0C94FF03CF93DF930E944511EC01E9
:10206000811522E59207E8F5811531E5930708F01F
:10207000B6C0883E910528F5803E910508F0E9C07C
:10208000883A910570F4853A910508F07AC081305C
:10209000910509F473C008F4D9C0049708F0D9C0B9
:1020A000D5C08F3B910508F0D1C0C85AD0E0CC0F05
:1020B000DD1FC25EDD4F0990D881C02DCE01946432
:1020C000C9C0811540E5940708F069C0811550E446
:1020D000950708F060C09A9581159F4108F4B9C032
:1020E000B5C0811536E5930728F5811545E59407B8
:1020F00008F092C0811554E5950708F087C0AC013F
:1021000043705527282F26952695C115D34508F0ED
:102110006CC081E090E002C0880F991F4A95E2F7F9
:1021200040E2249F90011124EC01C22BD32BCE015D
:102130009C6890C081152AE5920780F4811539E5E5
:10214000930708F072C0811548E5940708F47EC033
:10215000D82FCC27CE01806F906A7CC09056811515
:10216000904208F073C08D2F8F710E94D911DD2726
:10217000D0628F71AE01582BCA016CC081E090E033
:1021800069C0C55AD0E0C45BDD4F8881C82FD0E05C
:10219000CE0190645FC0DF70CE01906A5BC074E0D6
:1021A000969587957A95E1F7282F23703C2F337009
:1021B00081E090E002C0880F991F3A95E2F79C6891
:1021C000AC01522B9A019C2F9F709695969550E2E8
:1021D000959FE0011124C9018C2B9D2B3BC0D82F6A
:1021E000CC27CE01816F906A35C081E090E002C0BB
:1021F000880F991F4A95E2F750E2259F900111241C
:10220000EC01C22BD32BCE019A6824C0D82FCC2747
:10221000CE01846F906A1EC00E94D9118F7190E028
:10222000D82FCC27CE01906215C08F700E94D91193
:1022300094E0D695C7959A95E1F7CF70D0E0DC2F62
:10224000CC27D0699E01282BC90104C080E090E012
:1022500001C0CE01DF91CF9108952EE6829FC0018B
:102260001124FC012BE0729FE00DF11D1124E60FFB
:10227000F11DEE0FFF1FEC5DFE4F859194910895C7
:102280000E942D110E942B1008958238910569F14A
:10229000B0F48133910509F46DC048F48932910599
:1022A00009F463C08A32910509F469C00895853341
:1022B000910509F455C089339105B9F00895833E1D
:1022C000910569F138F4803E9105B1F0823E9105A7
:1022D00009F10895863E9105A9F1873E9105B9F16E
:1022E000843E910509F064C023C02091410420FD83
:1022F0004FC021FD4DC008958091410480FD44C030
:102300008091420480FF44C08091410484FD42C01A
:1023100083EE4DC08091410482FF38C0F5CF80919B
:10232000410482FD33C08091420480FD31C0ECCF76
:102330008091420481FF32C08091410484FD2AC013
:1023400087EE35C08091410483FF26C0F5CF809190
:10235000410483FD21C08091420481FD1FC0ECCF68
:102360008091410485FD1CC01DC08091410485FD04
:1023700019C016C08091410486FD16C017C0809117
:10238000410486FD13C010C089E311C082EE0FC066
:1023900080EE0DC080E00BC086EE09C084EE07C061
:1023A00089E205C085E303C08AE201C081E390E0D1
:1023B00008959091410492FF0DC0282F2871283074
:1023C00019F4877F846006C0282F2471243011F40B
:1023D0008B7F886093FF0DC0282F2871283119F456
:1023E000877E846106C0282F2471243111F48B7EEE
:1023F00088612091420420FF0DC0382F3871383099
:1024000019F4877F816006C0382F3171313011F4A3
:102410008E7F886021FF0DC0282F2871283119F484
:10242000877E816106C0282F2171213111F48E7EB3
:10243000886194FD877E089580E008950C94650E70
:102440000E9430138FE39CE90197F1F700C0000070
:102450000E94301380E00E945A1280FF04C00E9444
:102460001E120C94D92808950C9420120E946B0E11
:10247000811102C00E94130F0E94760E80934203C6
:102480000E947E0E90934204809341040E94341275
:102490000E947A0E682F70E080E090E00E9467084A
:1024A0006091CE027091CF028091D0029091D102C2
:1024B0000C949F08E82FF0E0EE0FFF1FE95AFB4F46
:1024C000808191810895089580EA8A95F1F70895B1
:1024D00000C008950C94641208950C946C120C942E
:1024E0006D120C946C120C947112F894E82FE29512
:1024F000EF70F0E031A1282F2F7081E090E001C053
:10250000880F2A95EAF7982F9095932391A392A18B
:10251000892B82A3789408950F931F93CF93DF9311
:10252000CAE5D2E089918F3F11F00E94751282E0D6
:10253000C436D807B9F7CFE4D2E00AE512E08991B2
:102540008F3F11F00E9475120C171D07C1F7DF9124
:10255000CF911F910F910895BF92CF92DF92EF928A
:10256000FF920F931F93CF93DF938C01C62FD0E080
:10257000CE01865A9D4F6C01FC0190819F3F09F46A
:1025800050C0B62EF894E92FE295EF70F0E081A1EB
:102590009F7021E030E001C0220F9A95EAF7822B6C
:1025A00081A382A12095282322A378940E946812F7
:1025B000EFE4F2E04AE552E021E030E0E12CF12CDA
:1025C00061916F3F89F0A62FA295AF70B0E0909611
:1025D0008C9190E06F7002C0959587956A95E2F7AF
:1025E00080FD02C0C90102C080E090E0E82AF92A1B
:1025F000220F331F4E175F0719F7F60180818F3FB7
:1026000011F00E94751261E0E114F10409F460E038
:102610008B2D0E946A12CC0FDD1FC00FD11FF982D3
:10262000E882DF91CF911F910F91FF90EF90DF90A3
:10263000CF90BF9008950E948C1284E1E7E5F4E00A
:10264000DF01982F1D929A95E9F7E3E4F4E0DF01AA
:102650001D928A95E9F78AE00E947B130C945E0331
:10266000FF920F931F93CF93DF93CDB7DEB764979D
:102670000FB6F894DEBF0FBECDBF8E010F5F1F4FA8
:1026800084E1F80111928A95E9F7F12C6F2DC801C8
:102690000E94AC12F394FAE0FF12F8CF44E150E04C
:1026A000B80183E494E00E948130FF24F394009702
:1026B00009F4F12C892B41F084E1F801A3E4B4E0A2
:1026C00001900D928A95E1F72F2D4AE067E574E0BD
:1026D00083E494E00E947C130E9460038F2D649633
:1026E0000FB6F894DEBF0FBECDBFDF91CF911F9123
:1026F0000F91FF9008950895FF920F931F93CF932A
:10270000DF93F82E092F162FD72FC42F222349F03D
:1027100081E0809345030E94702890934403809346
:102720004303809145038823D9F08091430390911E
:1027300044030E948828059798F0EF2DF02FA12FD1
:10274000BD2F80E090E04C2F50E08417950734F4C3
:10275000219131912D933D930196F7CF109245032E
:10276000DF91CF911F910F91FF9008950E94712AE0
:102770000E946E0F0C947D2A0E94812A0E941E10D6
:102780000C949B2A0E940E280E94582A0E94580FDF
:102790000E94B6130E94BC130E94620FFBCFEF92FF
:1027A000FF920F931F93CF93DF938B01682F11112B
:1027B0000AC0442329F0E82FF0E0E45AFC4F64916A
:1027C000762F862F75C0212F30E0E82FF0E04423CC
:1027D00021F0E45AFC4FE491F0E046E0049FC00190
:1027E0001124CFEFD0E0BE010E94BB2F4BEA46037D
:1027F000C001479F900D1124800F911D800F911DE6
:10280000982F990F890FAE01421B530B4E9FD00199
:102810004F9FB00D5E9FB00D11249B2F189FA001FC
:102820001124452F55278E01041B150B0E9FA00167
:102830000F9F500D1E9F500D11247E01E81AF108C4
:10284000E29E8001E39E100DF29E100D1124212FB7
:102850003327C21BD30BCE9F9001CF9F300DDE9F3D
:10286000300D112462307105A9F048F4611571052D
:1028700069F061307105C9F48B2F752F0DC064307C
:10288000710581F058F06630710579F47E2F8B2F39
:10289000932F0DC0832F7B2F9E2F09C08E2F7B2F50
:1028A000952F05C08E2F732F02C07E2F852F692F85
:1028B000DF91CF911F910F91FF90EF90089541E02C
:1028C0000E94CF13089520E030E0869F212D969F2F
:1028D000200D311D1124C9010895BC0182309105DC
:1028E00008F40895613E8EE1780748F49B0195E075
:1028F000369527959A95E1F748E0420F01C04FEFD2
:1029000091E0242F30E0290F311D35952795229F26
:10291000F001239FF00DF00D11246E177F0718F4BE
:102920004FEF420F04C02F3F39F091E0920F49174B
:1029300040F78FEF890F08958FEF08954091D901E7
:102940005091DA0125E038E0429FC001439F900D8D
:10295000529F900D1124875E994C9093DA018093D9
:10296000D901890F0895482F982F46FD9095E92F9A
:10297000EF739F7046FD9F5FE295EF70EE0FF0E002
:10298000EC59FD4F2181299F802D212D1124829505
:102990008F702295207F822B3081982F930F892F63
:1029A00047FD819580580895E42FF0E0EE0FFF1F5A
:1029B000EE58FE4F408134EE439F412D1124E72F06
:1029C000F0E050E0445E5F4FDA01A21BB1099D01C7
:1029D000B7FF03C031952195310993E0220F331FD2
:1029E0009A95E1F7AF01421B530B9A0157FF02C0C2
:1029F00020E030E0279F212D1124722F0895E42F2D
:102A0000F0E0EE0FFF1FEE58FE4F408134EE439F83
:102A1000412D1124E82FF0E050E0445E5F4FDA01D1
:102A2000A21BB1099D01B7FF03C031952195310962
:102A300093E0220F331F9A95E1F7AF01421B530B2E
:102A40009A0157FF02C020E030E0582F259F212D2A
:102A50001124822F0895622F0895E42FF0E0EE0FE5
:102A6000FF1FEE58FE4F6081621B0895E42FF0E0D7
:102A7000EE0FFF1FED58FE4F6081621B0895A22FDD
:102A800050E0FA01EE0FFF1FED58FE4F908190527B
:102A900097FD9195440F551FFA01EE58FE4F308176
:102AA000232F30E02A1B3109290F311D97FD3A955C
:102AB000620F0895EF920F931F9393E0099F800197
:102AC0001124159507956E2D600F1F910F91EF90B2
:102AD00008950F93CF93DF93D72FC82F47FD4195CC
:102AE000E8E3F0E0CF01841B910947FD9395889FAF
:102AF000B001899F700D700D1124229FC001239F8A
:102B0000900D900D1124860F971F0E946D14682F51
:102B1000660F860F682F600F7D2F8C2FDF91CF916E
:102B20000F9108950F931F93522F10E0F801EE0FAD
:102B3000FF1FED58FE4FE081F0E0B0979F01520378
:102B4000D001539FB00D1124000F111FF801EE5852
:102B5000FE4F008110E00057110940039001419F92
:102B6000300D11242A0F3B1F37FF02C021583F4F61
:102B7000220F232F221F330B620F1F910F910895F5
:102B80000F931F93522F10E0F801EE0FFF1FED5827
:102B9000FE4FE081F0E0B097EE0FFF1F9F01520360
:102BA000D001539FB00D1124000F111FF801EE58F2
:102BB000FE4F008110E000571109000F111F400364
:102BC0009001419F300D11242A0F3B1F37FF02C097
:102BD00021583F4F220F232F221F330B620F1F91CB
:102BE0000F9108950F931F9310E0F801EE0FFF1F50
:102BF000EE58FE4F9081905797FD9195000F111F51
:102C0000F801ED58FE4FE081F0E0B097DF01AA0F28
:102C1000BB1F8D010E0F1F1F2003D001219FB00D80
:102C20001124E8E3F0E0E91BF10997FDF3959F011A
:102C3000220F331F89010E0F1F1F40039001419F78
:102C4000300D11242A0F3B1F37FF02C021583F4F80
:102C5000220F232F221F330B620F1F910F91089514
:102C60000F931F93CF93DF93D62F072F182FC42FC7
:102C7000822F0E94B314EC2FF0E0EE0FFF1FEE58EE
:102C8000FE4F90819058890F87FD8195880F682F9E
:102C90002CE0629F612D11246D0F702F812FDF9129
:102CA000CF911F910F910895E42FF0E0EE0FFF1FD9
:102CB000EE58FE4F9081921B97FD9195292F38E198
:102CC000239F212D1124620F089520916F0430E17C
:102CD000230F08F42FEF60E1822F90E00E9463142D
:102CE000BC0188EB9BE00E94BB2F80E090E0089540
:102CF000FC019B01009721F477FF2BC080E8089529
:102D0000AC0197FF04C044275527481B590BB90154
:102D1000640F751F37FD0CC0241B350BC901A5E0DE
:102D2000880F991FAA95E1F70E94CF2F80E20CC06F
:102D3000CB0165E0880F991F6A95E1F7BA01621B24
:102D4000730B0E94CF2F80E6861BF7FF03C081958F
:102D5000089580E00895FF920F931F93CF93DF9320
:102D6000F62E172FD82FC901C72FC01BBA010E94FA
:102D70007816982F990F890F7C2F781B719F712DD2
:102D800011246F2D8D2FDF91CF911F910F91FF9007
:102D90000895FF920F931F93CF93DF93F62ED72FB3
:102DA000182FC901C12FC01BBA010E947816982F95
:102DB000990F890FC81B2C2F219F212D1124822FA1
:102DC0006F2D7D2FDF91CF911F910F91FF9008956F
:102DD000EF920F931F93CF93DF93D62F172FC82F08
:102DE000C9010E19070FBA010E947816702F781BBF
:102DF000719F712D11246D2F8C2FDF91CF911F9119
:102E00000F91EF900895EF920F931F93CF93DF935D
:102E1000D62FC72F182FC9010E19010FBA010E9412
:102E20007816081B202F219F212D1124822F6D2F12
:102E30007C2FDF91CF911F910F91EF9008950F9309
:102E4000CF93DF93D72FC82FC901BA010E947816FC
:102E5000682F600F7D2F8C2FDF91CF910F910895F8
:102E6000EF920F93CF93DF93D72FC82FC9010E197D
:102E7000BA010E947816602F681B7D2F8C2FDF917E
:102E8000CF910F91EF9008950E945F140895EBE6A3
:102E9000F4E085E380838091EA019091EB01A091B9
:102EA000EC0181839283A3838FE784838FEF8583F3
:102EB00046E050E06CE170E0CF010E94AC3010922F
:102EC0001D040895E0917202F09173020994E0915B
:102ED0006E02F0916F0209944F925F926F927F920F
:102EE0008F929F92AF92BF92CF92DF92EF920F9309
:102EF0001F93CF93DF932C013B01FC01C08187E03E
:102F0000C89FC02D1124D7E0DC0FD03208F0DFE1DC
:102F100060916F04669580917104909172040E9493
:102F20006314182FCD1708F044C08C2E912CF40197
:102F3000E055FE4F9081F20181818923C1F1F401B6
:102F4000EE0FFF1FEE58FE4FC080D12CF0E7CF1AD6
:102F5000D108F401EE0FFF1FED58FE4FA080B12CF9
:102F600080E2A81AB108CC9C9001CD9C300D300DA8
:102F70001124AA9CC001AB9C900D900D1124820FCE
:102F8000931F0E946D14082F60916C0470916D0462
:102F900080916E04E12E9501A601F30109950E942E
:102FA0004417462F282F672FC4010E946717CF5F51
:102FB000B9CF81E0DF3108F080E0DF91CF911F9140
:102FC0000F91EF90DF90CF90BF90AF909F908F9038
:102FD0007F906F905F904F90089568EE76E10C942B
:102FE0006C1763E077E10C946C176AE575E10C945B
:102FF0006C1760E377E10C946C17AF92BF92CF929D
:10300000DF92EF92FF920F931F93CF93DF936C01A8
:103010005B01FC01C08187E0C89FC02D1124D7E06F
:10302000DC0FD03208F0DFE160916F04669580918B
:103030007104909172040E946314182FCD1778F5D3
:10304000EC2EF12CF701E055FE4F9081F6018181C5
:10305000892319F1F701EE0FFF1FED58FE4F208174
:1030600030E020523109F701EE0FFF1FEE58FE4FFE
:10307000408150E04057510960916C0470916D049B
:1030800080916E04012FF50109950E944417462F87
:10309000282F672FC7010E946717CF5FCFCF81E02E
:1030A000DF3108F080E0DF91CF911F910F91FF9009
:1030B000EF90DF90CF90BF90AF9008956BEA76E1EC
:1030C0000C94FD1769EC76E10C94FD1769E675E147
:1030D0000C94FD176FE177E10C94FD17BF92CF922E
:1030E000DF92EF92FF920F931F93CF93DF938C01A8
:1030F0007B01FC01C08187E0C89FC02D1124D7E06F
:10310000DC0FD03208F0DFE160916F0466956695C0
:1031100021E0620F08F46FEF8091710490917204C6
:103120000E946314B82ECD17F0F4CC2ED12CF601EA
:10313000E055FE4F9081F8018181892391F06091E3
:103140006C0470916D0480916E042B2D4C2FF7014F
:1031500009950E944417462F282F672FC6010E9409
:103160006717CF5FE0CF81E0DF3108F080E0DF91CB
:10317000CF911F910F91FF90EF90DF90CF90BF9074
:10318000089564ED74E10C946E186FEF74E10C9483
:103190006E186BE275E10C946E186DE275E10C949B
:1031A0006E1866E375E10C946E186FE375E10C948C
:1031B0006E1860E376E10C946E1864E576E10C9489
:1031C0006E187F928F929F92AF92BF92CF92DF92B2
:1031D000EF92FF920F931F93CF93DF936C015B01EC
:1031E000FC01C08187E0C89FC02D1124D7E0DC0F0F
:1031F000D03208F0DFE160916F04669566958091AA
:103200007104909172040E946314182F80E4810F5E
:103210000E94B31490E8F92EF80E812F0E94B31487
:1032200020E8722E780ECD1700F58C2E912CF4012B
:10323000E055FE4F9081F60181818923A1F06091D4
:103240006C0470916D0480916E04E12E0C2F272D7B
:103250004F2DF50109950E944417462F282F672FFF
:10326000C4010E946717CF5FDECF81E0DF3108F035
:1032700080E0DF91CF911F910F91FF90EF90DF9051
:10328000CF90BF90AF909F908F907F90089562E90C
:1032900075E10C94E11860EC75E10C94E11862EFB3
:1032A00075E10C94E118DF92EF92FF920F931F9358
:1032B000CF93DF938C01DC018C91C7E08C9FC02DF4
:1032C0001124D7E0DC0FD03208F0DFE160916C040C
:1032D00070916D0480916E040E944417F62EE72EC3
:1032E000D82ECD1798F4EC2FF0E0DF01A055BE4F9B
:1032F0008C91D80111969C91982331F02D2D4F2D52
:103300006E2DCF010E946717CF5FEBCF81E0DF31D9
:1033100008F080E0DF91CF911F910F91FF90EF9027
:10332000DF900895AF92BF92CF92DF92EF92FF921B
:103330000F931F93CF93DF938C01FC01C08187E033
:10334000C89FC02D1124D7E0DC0FD03208F0DFE198
:10335000E0906D04F0906E04D0906C046D2D7E2D85
:103360008F2D0E944417C62EB72EA82E60916F0491
:103370006D0D7E2D8F2D0E944417F62EE72ED82E30
:10338000CD17B8F48C2F90E0FC01E055FE4F308152
:10339000F8012181232359F030FF04C02D2D4F2D3A
:1033A0006E2D03C02A2D4C2D6B2D0E946717CF5F09
:1033B000E7CF81E0DF3108F080E0DF91CF911F910E
:1033C0000F91FF90EF90DF90CF90BF90AF90089556
:1033D000BF92CF92DF92EF92FF920F931F93CF9302
:1033E000DF936C01FC01C08187E0C89FC02D1124D0
:1033F000D7E0DC0FD03208F0DFE100916D04B0902F
:103400006E0420916F0410E4129F112D1124CD172A
:1034100018F5EC2EF12CF701E055FE4F9081F601E6
:1034200081818923B9F0F701EE0FFF1FED58FE4FA0
:10343000808182958F7060916C04819F600D112452
:10344000702F8B2D0E944417462F282F672FC701FE
:103450000E946717CF5FDBCF81E0DF3108F080E0AB
:10346000DF91CF911F910F91FF90EF90DF90CF9060
:10347000BF900895BF92CF92DF92EF92FF920F9389
:103480001F93CF93DF937C01FC01C08187E0C89F2D
:10349000C02D1124D7E0DC0FD03208F0DFE1C0905E
:1034A0006D04B0906E0420916F0430E4D32E3D2D56
:1034B000329F312D1124D32ECD1738F50C2F10E06B
:1034C000F801E055FE4F9081F70181818923D9F001
:1034D000F801EE0FFF1FEE58FE4F6081D69EB0013F
:1034E000112495E0759567959A95E1F780916C04A4
:1034F000680F7C2D8B2D0E944417462F282F672F95
:10350000C8010E946717CF5FD7CF81E0DF3108F095
:1035100080E0DF91CF911F910F91FF90EF90DF90AE
:10352000CF90BF900895DF92EF92FF920F931F9379
:10353000CF93DF938C01DC01CC9187E0C89FC02D35
:103540001124D7E0DC0FD03208F0DFE1E0906C040A
:10355000F0906D04D0906E0460916F04669566954E
:10356000669580917104909172040E9463140E9488
:10357000B314805887FD8195880F282F3D2D239FF8
:10358000212D1124822FB7010E944417F62EE72E19
:10359000D82ECD1798F4EC2FF0E0DF01A055BE4FE8
:1035A0008C91D80111969C91982331F02D2D4F2D9F
:1035B0006E2DCF010E946717CF5FEBCF81E0DF3127
:1035C00008F080E0DF91CF911F910F91FF90EF9075
:1035D000DF900895DF92EF92FF920F931F93CF93A6
:1035E000DF93EC01FC01E055FE4F9081692381F1EE
:1035F000D0906D0400916E0410916C04E12EF12CBA
:103600000E947130282FC7018C549F4F68E671E0EB
:103610000E94CF2F8E199F0997FD03969595879548
:10362000959587952370612F289F600D11247D2D1E
:10363000802F0E944417462F282F672FCE01DF913D
:10364000CF911F910F91FF90EF90DF900C9467172F
:10365000DF91CF911F910F91FF90EF90DF90089530
:10366000CF92DF92FF920F931F93CF93DF938C0142
:10367000FC01C281C1111DC060916F0420E1620F85
:1036800008F46FEF80917104909172040E946314AA
:103690006AE070E00E94BB2F892B59F50E947130BF
:1036A0006FE170E00E94CF2FF80161810E94EA1A59
:1036B00020C0FC018081C7E08C9FC02D112497E0C1
:1036C000F92EFC0EFFE1FF1510F48FE1F82ED0E08B
:1036D000CF2CD12CCC15DD053CF4F8016181CE0155
:1036E0000E94EA1A2196F6CFC1E0FEE1FF1508F428
:1036F000C0E08C2FDF91CF911F910F91FF90DF9051
:10370000CF9008951F93CF93DF93FC01E055FE4FB8
:1037100020816223D1F0EC010E947130182F0E94A9
:1037200071308F77782F20E8720F08F47FEF612FC8
:1037300080916E040E944417462F282F672FCE01D8
:10374000DF91CF911F910C946717DF91CF911F915B
:103750000895CF92DF92FF920F931F93CF93DF9341
:103760008C01FC01C281C1111DC060916F0420E178
:10377000620F08F46FEF80917104909172040E94BF
:10378000631465E070E00E94BB2F892B59F50E94FD
:1037900071306FE170E00E94CF2FF80161810E94CB
:1037A000821B20C0FC018081C7E08C9FC02D1124AA
:1037B00097E0F92EFC0EFFE1FF1510F48FE1F82ED3
:1037C000D0E0CF2CD12CCC15DD053CF4F801618183
:1037D000CE010E94821B2196F6CFC1E0FEE1FF15CB
:1037E00008F4C0E08C2FDF91CF911F910F91FF90D3
:1037F000DF90CF900895DF92EF92FF920F931F9387
:10380000CF93DF938C01DC01CC9187E0C89FC02D62
:103810001124D7E0DC0FD03208F0DFE1E0906D0436
:10382000F0906E04D0906C0460916F04669566957C
:10383000669580917104909172040E9463140E94B5
:10384000B314805887FD8195880F682F2CE0629F04
:10385000612D11246D0D7E2D8F2D0E945F14F62E8B
:10386000E72ED82ECD1798F4EC2FF0E0DF01A0550D
:10387000BE4F8C91D80111969C91982331F02D2D3B
:103880004F2D6E2DCF010E946717CF5FEBCF81E0E8
:10389000DF3108F080E0DF91CF911F910F91FF9011
:1038A000EF90DF900895E0917002F0917102099419
:1038B0000C94470F08950C945A1C0E945B1C0C94A6
:1038C000F40208950C94611CCF93DF93FC01C08136
:1038D000C15087E0C89FC02D1124D7E0DC0FD03243
:1038E00008F0DFE16D2F8C2F0E94621C6D2F8C2F52
:1038F000DF91CF910C94611C5F926F927F928F92B7
:103900009F92AF92BF92CF92DF92EF92FF920F936E
:103910001F93CF93DF930E947C2860931E047093C3
:103920001F04809320049093210430916B04232F73
:10393000237021F0F32EF694F69401C0F12C20911F
:10394000D301213091F028F0223091F12330E1F1C0
:1039500032C31092D4016093710470937204809307
:1039600073049093740481E02CC09091D701F912F4
:103970000DC0832F837090E04091D80150E021E08A
:103980008417950709F420E0822F01C081E081703F
:103990008093D601809170049091D5019817A9F178
:1039A0008093D50140E060E080E00E94531C2DC070
:1039B000F092D701832F83708093D8010E94621701
:1039C00083E08093D301F7C280911D04882351F0D6
:1039D00046E050E06CE170E08BE694E00E94AC3091
:1039E00010921D04609171047091720480917304AF
:1039F000909174040E9497286031710581059105AA
:103A000008F4D9C21092D301D6C28F2D90E08F3125
:103A1000910598F18091D4018F5F8093D40182E069
:103A20008093D3018091D601811123C0FF2041F200
:103A30000E945D1C84ED91E0DF91CF911F910F9169
:103A4000FF90EF90DF90CF90BF90AF909F908F90BE
:103A50007F906F905F900C94641C84ED91E00E94C5
:103A60005319C82F8091D4018F5F8093D401CC2348
:103A7000B1F2FF2009F49FC2DBCFFC01EE59FF4FEA
:103A80000C9405308091D601882309F492C240E05D
:103A900060E080E00E94531C8CC284ED91E00E94A3
:103AA0009219DFCF84ED91E00E94E819DACF84ED1E
:103AB00091E00E943A1AD5CF84ED91E00E94931ACA
:103AC000D0CF84ED91E00E94C118CBCF84ED91E07E
:103AD0000E94C518C6CF84ED91E00E945E18C1CF48
:103AE00084ED91E00E946218BCCF84ED91E00E94C9
:103AF000ED17B7CF84ED91E00E94F117B2CF84EDBE
:103B000091E00E94C918ADCF84ED91E00E94CD18DC
:103B1000A8CF84ED91E00E94D118A3CF84ED91E06D
:103B20000E94D5189ECF84ED91E00E94F51799CFA1
:103B300084ED91E00E94661894CF84ED91E00E949C
:103B40006A188FCF84ED91E00E94F9178ACF84ED37
:103B500091E00E94471985CF84ED91E00E944B19B6
:103B600080CF84ED91E00E944F197BCF84ED91E0EE
:103B70000E94301B76CF84ED91E00E94A91B71CF8B
:103B800084ED91E00E94FB1B6CCF84ED91E00E94DC
:103B9000D91867CF84ED91E00E94DD1862CF409183
:103BA000190450911A0460911B0470911C048091B7
:103BB000710490917204A0917304B09174048417FD
:103BC0009507A607B70708F4F4C10E949E14182FA2
:103BD0000E949E149FE1891BF0F7890FC82FD0E047
:103BE000FE01E055FE4F9091D5018081892309F4B3
:103BF000DEC111FF04C020E040E060E013C00E947D
:103C00009E14182F0E949E148695782F2FE7720F0E
:103C100008F47FEF612F80916E040E944417462FB5
:103C2000282F672FCE010E94671720916F0430E183
:103C3000230F08F42FEF60E1822F90E00E946314BD
:103C4000BC0184EF91E00E94BB2F809171049091A0
:103C50007204A0917304B0917404860F971FA11D84
:103C6000B11D8093190490931A04A0931B04B09380
:103C70001C049FC1409115045091160460911704D3
:103C8000709118048091710490917204A091730452
:103C9000B091740484179507A607B70708F489C183
:103CA0008091D60181110DC08091D401C7E08C9F15
:103CB000C02D112407E00C0F003208F451C00FE1B1
:103CC0004FC040E060E080E00E94531C08EB13E02E
:103CD000C0E0D0E0FFE7EF2E0E949E1481FF05C0F8
:103CE000F8011082118212821DC00E949E14B82E0B
:103CF0000E949E148695782F2E2D720F08F47FEF68
:103D0000CE01880F991F8C0F9D1FFC01E854FC4FBA
:103D10006F016B2D80916E040E945F14F601608329
:103D20007183828321960D5F1F4FCF31D105A1F69C
:103D3000BBCF8C2F90E0FC01E055FE4F30812091ED
:103D4000D501232361F0FC01EE0FFF1FE80FF91FDF
:103D5000E854FC4F2281408161810E946717CF5F48
:103D6000C01738F3C1E00F3108F0C0E00F3108F49C
:103D700079CE20E010E001501109822F90E08017E9
:103D80009107CCF4AC01440F551F480F591F4854FC
:103D90005C4F0196FC01EE0FFF1F8E0F9F1FFC0171
:103DA000E854FC4F80819181A281FA018083918344
:103DB000A2832F5FE2CF0E949E146801CC0CDD1C11
:103DC00081FF09C00C0D1D1DF801E854FC4F108245
:103DD0001182128218C00E949E14D82F0E949E1435
:103DE0008695782F2FE7720F08F47FEF0C0D1D1DBD
:103DF00008541C4F6D2F80916E040E945F14F801CF
:103E00006083718382830E94651600917104109112
:103E100072042091730430917404DC01CB01800F93
:103E2000911FA21FB31F8093150490931604A093B3
:103E30001704B093180416CE4091B4035091B50303
:103E40006091B6037091B7038091710490917204F0
:103E5000A0917304B091740484179507A607B7075F
:103E600008F4A7C08091D601882329F040E060E0E3
:103E700080E00E94531C60916C0470916D048091ED
:103E80006E040E944417E62E772E682EC6E4D3E017
:103E900004E011E094EBA92E93E0B92E48016E01E5
:103EA000512CF6018081F401882329F08081262D90
:103EB0004E2D672D04C0808120E040E060E090E05E
:103EC0000E946717F601818181936F015394FFEF80
:103ED0008F1A9F0A24E05212E4CF48016E018AE053
:103EE000582EF6018285F401882329F08285262D3B
:103EF0004E2D672D04C0828520E040E060E090E018
:103F00000E946717F601818582875A94F1E0CF1AE3
:103F1000D10821E0821A910835E05312E2CF8D8159
:103F2000F801882329F08581262D4E2D672D04C0A8
:103F3000858120E040E060E090E00E9467178C817E
:103F4000F801882329F08481262D4E2D672D04C089
:103F5000848120E040E060E090E00E9467170E94CA
:103F60009E14837091E009F090E09C839D832B96D2
:103F7000055F1F4FAC16BD0609F090CF0E94651675
:103F800000917104109172042091730430917404B3
:103F9000DC01CB01800F911FA21FB31F8093B403DC
:103FA0009093B503A093B603B093B70302C0C1E0EA
:103FB00059CDC0E057CDDF91CF911F910F91FF9068
:103FC000EF90DF90CF90BF90AF909F908F907F90B9
:103FD0006F905F900895E0916C02F0916D020995E9
:103FE0000E946B0E811104C00E94130F0E9447179C
:103FF00046E050E06CE170E08BE694E00E948E3089
:1040000010921D0480916B048C7F11F40C9447175F
:1040100008950895EBE6F4E0208191E092279083E3
:104020001092D30190911D04892B80931D04089553
:1040300081E00C940A2090916B049370A1F081119F
:1040400002C0946007C08F3110F0986703C0880FDA
:10405000880F982B90936B041092D30180911D04CC
:10406000682B60931D04089561E00C941B20682F59
:1040700090916B04969596959F5F9F3110F4892FD0
:1040800001C081E00C941B2081E00C943720682F44
:1040900090916B0496959695915011F0892F01C0DF
:1040A0008EE10C941B2081E00C94472090916B04CE
:1040B000937059F080936C0460936D0440936E0488
:1040C00080911D04282B20931D040895ABE6B4E0D5
:1040D0001196EC911197F0E0282F13964C911397BD
:1040E00012966C91CF0108960C94562081E00C94A6
:1040F0006620ABE6B4E01196EC911197F0E0282F22
:1041000013964C91139712966C91CF0108970C94CB
:10411000562081E00C947920EBE6F4E0628120E106
:10412000620F08F46FEF9181282F4381892F90E06F
:104130000C94562081E00C948C20EBE6F4E0628134
:1041400020E1621B08F460E09181282F4381892FD0
:1041500090E00C94562081E00C949D20EBE6F4E076
:10416000438120E1420F08F44FEF9181282F6281B3
:10417000892F90E00C94562081E00C94AE20EBE661
:10418000F4E0438120E1421B08F440E09181282FB4
:104190006281892F90E00C94562081E00C94BF201E
:1041A00080936F0480911D04682B60931D04089513
:1041B00020916F0430E1230F08F42FEF682F822F36
:1041C0000C94D02081E00C94D82020916F0430E131
:1041D000231B08F420E0682F822F0C94D02081E06C
:1041E0000C94E5200895FC01EE0FFF1F8E0F9F1F1A
:1041F000FC01EB58FB4F6183408322830895E5E780
:10420000F4E094E0E23DF90729F081836083428382
:104210003396F7CF08956FE170E085E794E00C9452
:104220006524882311F0FA0101C0FB0109941F9352
:10423000CF93DF93FB011281111191C0EC010E9419
:10424000820D8272CB3CFCE5DF0709F472C010F5E9
:10425000C63CECE5DE0709F453C058F4C43C9CE5C9
:10426000D90709F441C008F044C0C33CDC45C9F19A
:1042700036C0C83C9CE5D90709F44CC008F445C0D9
:10428000C93CFCE5DF0709F44AC0CA3CDC4509F437
:104290004BC025C0C03DECE5DE0709F45DC088F4E5
:1042A000CD3C9CE5D90709F44EC008F447C0CE3C8C
:1042B000FCE5DF0709F44CC0CF3CDC4509F44AC0FB
:1042C0000EC0C73D9CE5D90730F4C23DDC4508F07F
:1042D00046C082E142C0CE35DD4509F440C011E060
:1042E0003EC00E9418203BC043E550E264E470E207
:1042F00004C044E450E263E570E20E9411212FC043
:1043000049E850E266E770E2F8CF46E750E269E834
:1043100070E2F3CF4BEA50E26AE970E2EECF4AE98D
:1043200050E26BEA70E2E9CF4DEC50E26CEB70E2E8
:10433000E4CF4CEB50E26DEC70E2DFCF4FEE50E299
:1043400062EE70E2DACF42EE50E26FEE70E2D5CF6D
:1043500081E003C085E001C08DE00E943420812F00
:10436000DF91CF911F91089586E090E00C949E30EC
:10437000682F86E090E00C94BC308091D204847069
:1043800081628093D2040C94B8218091D2048695E6
:104390008695869508958091D20481FD07C082603C
:1043A0008093D2040E94B8210C94B4230895809184
:1043B000D20481FF07C08D7F8093D2040E94B82170
:1043C0000C94C02308958091D20481FD0C94D721D0
:1043D0000C94CB218091D2048695817008958091B0
:1043E000DB0108950E946B0E811104C00E94130F1F
:1043F0000E94BD210E94B4218093D204282F2695CB
:104400002695269530E02530310524F087708062AE
:104410008093D2048091D20480FF04C08695869553
:10442000869501C080E00C9486232091D204822FCF
:10443000869586958695482F50E04430510554F472
:104440008F5F982F990F990F990F822F8770892B63
:104450008093D2048091D20481608093D2040E9420
:10446000B8218091D2048695869586950C948623F2
:104470008091D204982F969596959695A1F0915E8D
:10448000990F990F990F8770892B8093D204887F99
:1044900091E009F490E08091D20490FB80F9809340
:1044A000D2040E94B8218091D20486958695869583
:1044B0000C9486238091D20480FD13C08160809388
:1044C000D204813019F489E08093D2048091D2041F
:1044D0000E94B8218091D2048695869586950C9489
:1044E000862308958091D20480FF08C08E7F809338
:1044F000D2040E94B82180E00C9486230895809114
:10450000D20480FD0C9472220C945A229091D20411
:10451000892F8695869586958F5F8F7197708530E8
:1045200038F4880F880F880F892B8093D20402C03B
:104530009093D2048091D204887F91E009F490E0B6
:104540008091D20490FB80F98093D2040E94B8211C
:104550008091D2048695869586950C948623853025
:1045600008F084E09091D2049770282F220F220F38
:10457000220F922B9093D204987F21E009F420E03F
:104580009091D20420FB90F99093D2040C9486234E
:104590000E94AF228091D2040C94B821FC01DB016F
:1045A00012968C918823F9F0EC5BFC45E730F1051D
:1045B000D8F4EF57FF4F0C94053084E001C080E041
:1045C0000E94C82280E008950E943822FBCF0E94FA
:1045D0001522F8CF0E947F22F5CF0E948622F2CFCB
:1045E0000E94E321EFCF81E00895279A2F98089544
:1045F0002F9808958F929F92AF92BF92CF92DF92A1
:10460000EF92FF920F931F93CF93DF938C018091D2
:104610008600909187006CE070E00E94BB2F6017CD
:10462000710730F0C80169E070E00E94BB2F60C0E4
:104630008091860090918700E0908600F09087003E
:10464000E0918600F0918700C6E0D0E0BE010E94B4
:10465000BB2F20E030E0060F171F211D311D480140
:10466000590185E0880C991CAA1CBB1C8A95D1F7BE
:10467000C701BE010E94BB2F6F01E12CF12CA701E5
:104680009601260F371F411D511DC501B4010E941F
:10469000E32F69017A01E0918600F0918700CA0159
:1046A000B9010E94AB2F9B01AC01DF010E941A30BF
:1046B0009B01AC01C701B6010E94AB2FDC01CB010D
:1046C0002FE0B695A795979587952A95D1F70091F4
:1046D00086001091870020E030E0081719072A07AC
:1046E0003B0728F46091860070918700CB01BC01E4
:1046F000CB01DF91CF911F910F91FF90EF90DF9051
:10470000CF90BF90AF909F908F900895CF93C82F78
:10471000853050F4811109C080918000877F80939B
:1047200080000E94F82206C0C4E08091800088606A
:1047300080938000A0918600B09187002C2F30E0FC
:104740000E940B30DC01CB0122E0B695A79597952E
:1047500087952A95D1F70E94FA2290938D00809335
:104760008C00CF9108950895109223041092220492
:1047700010922404EFE6F0E0808181608083089548
:10478000EFE6F0E080818E7F80830E94C5210C944B
:1047900086231F920F920FB60F9211240F931F932F
:1047A0002F933F934F935F936F937F938F939F9339
:1047B000AF93BF93CF93EF93FF938091DC0191E090
:1047C000980F823019F09093DC0155C081E08093FE
:1047D000DC010E94EF21C82F0091220410912304D4
:1047E0000F5F1F4F0E94EF2128E7829FB001112425
:1047F000C8010E94BB2F909323048093220428E7D2
:10480000C29FB0011124660F672F661F770B719549
:104810000E94BB2F6F7780912404823019F460349A
:1048200051F404C0813039F46F3729F480916F005E
:104830008E7F80936F00E62FF0E0E452FD4FC4912D
:1048400000918600109187000E94C521282FC09FEB
:10485000C001C19F900D11246CEF73E00E94BB2F2B
:10486000269FC001279F900D11240E94FA22909349
:104870008D0080938C00FF91EF91CF91BF91AF910C
:104880009F918F917F916F915F914F913F912F9168
:104890001F910F910F900FBE0F901F9018950E94BF
:1048A000F5228AE08093800089E1809381008FEF78
:1048B0009FEF90938700809386000E94F2210E94D0
:1048C000EA2181110C94B42308956A9A2EB12B7FAA
:1048D0003EB134604FB7F894FC01CB01880F991FAB
:1048E000680F791F6E0F7F1FE617F70789F0819118
:1048F00098E03EB9000000C087FF2EB9880F000085
:1049000000C000C000C02EB900C09A9591F7ECCF4E
:104910004FBF8FE594E00197F1F700C000000895C4
:10492000CF93DF93EC01FB018281882309F43CC122
:10493000C430FDE5DF0760F4CB3F9CE5D90788F480
:104940009E0122503C452431310508F02EC109C09A
:10495000C236EDE5DE0729F0C63AFDE5DF0709F0CE
:1049600024C10E947E0E9093420480934104C13181
:104970008CE5D80709F4C6C008F042C0C930ECE5A0
:10498000DE0709F49BC000F5C5308CE5D80709F4B3
:1049900085C078F4C330ECE5DE0709F478C008F090
:1049A0007AC0C230DC4509F0F5C0809141048160D5
:1049B000EFC0C7309CE5D90709F478C008F07AC089
:1049C000809141048061E4C0CD30FCE5DF0709F44B
:1049D00087C058F4CB309CE5D90709F479C008F0BA
:1049E0007BC08091410488606FC0CF30FCE5DF0759
:1049F00009F480C008F082C080914104877FC8C05C
:104A0000CE3F9CE5D90709F471C000F5C531FCE53E
:104A1000DF0709F485C068F4C3319CE5D90709F4C0
:104A200075C008F095C00E940F08809141048F77EF
:104A3000AFC0CC3FFCE5DF07A9F108F054C0CB3F85
:104A4000DC4509F0A7C08091420440C0C230EDE5CA
:104A5000DE0709F489C058F4C1158DE5D80709F4BB
:104A60005AC008F069C08091420482602FC0C236EB
:104A7000EDE5DE0709F47CC0C63AFDE5DF0709F481
:104A800081C0C330DD4509F085C080E06EC08091F3
:104A9000410482607DC08091410416C08091410430
:104AA000886076C08091420482604FC0809141044A
:104AB00080626EC08091410480646AC00E940F08C9
:104AC00080914104806864C0846062C081603DC0A0
:104AD000809141048E7F5CC0809141048D7F58C0DD
:104AE0008091410416C08091420418C08091420414
:104AF0008D7F2BC0809141048F7E4AC080914104FC
:104B00008F7D46C0809141048F7B42C080914104DB
:104B1000877F8B7F3DC0809142048D7F8E7F15C043
:104B20008091410482FB222720F991E0922790FB9B
:104B300082F990FB83F92CC080914204982F9095C4
:104B400091708E7F892B90FB81F98093420422C063
:104B50000E940F088091410487FB222720F991E0F1
:104B6000922790FB87F914C081E00E94150F12C0B4
:104B70008091410484FB222720F991E0922790FB49
:104B800084F906C080914104982F909590FB80F99C
:104B90008093410480914104909142040E948F0EC1
:104BA0000E940F0880E001C081E0DF91CF9108955D
:104BB0008FE891E00197F1F700C0000008950C9490
:104BC000DB0222982A9A23982B9A0E94D82583B137
:104BD00082FB882780F91B9902C090E001C092E017
:104BE000892B809327040895E0912704EE0FEE0FA0
:104BF000E093270443B142FB882780F990E043B15A
:104C000043FB222720F930E043FF02C022E030E0DE
:104C1000822B932B8E2B809327048F70E82FF0E04C
:104C2000EC58FD4F908180912604890F80932604D3
:104C300084305CF0809125048F5F8093250460E0D0
:104C400080E00E94DF2521E001C020E08091260461
:104C50008D3F54F48091250481508093250461E0B8
:104C600080E00E94DF2521E080912604082E000CC0
:104C7000990B64E070E00E94CF2F80932604822F6E
:104C80000895CF93DF9386319C4541F5EB010E9457
:104C9000820D982F8A812091D1013091D2018823F1
:104CA00079F09A7A81E009F480E0809328049111E8
:104CB00002C069E201C065E3C9010E94C9270AC0B8
:104CC00080912804811102C069E201C065E3C90135
:104CD0000E94CB270E94C40D80E001C081E0DF91DB
:104CE000CF9108950F931F93CF93DF93C42FD22FAB
:104CF000FC0182818823C9F040932B040E94702814
:104D000090932A048093290480E28C0F883008F065
:104D100057C0C77081E001C0880FCA95EAF7DF91DC
:104D2000CF911F910F910C947B0580912B04481318
:104D300030C08091290490912A040E948828883CE0
:104D4000910538F510E21D0FCD17B9F080E28C0FF8
:104D5000883040F4C77081E001C0880FCA95EAF737
:104D60000E948205183028F581E09D2F977001C0C0
:104D7000880F9A95EAF70E947B05802F0E947205A2
:104D80001830F0F4D77081E001C0880FDA95EAF7A7
:104D90000AC080E28C0F883098F4C77081E001C0AF
:104DA000880FCA95EAF7DF91CF911F910F910C946C
:104DB0008205802FDF91CF911F910F910C94720586
:104DC000DF91CF911F910F9108950F939C01CB011B
:104DD000243F4CE5340731F188F4293DFCE53F07D9
:104DE000D9F02A3D4CE5340779F1283D3C45A9F539
:104DF00006E221EE41EE68ED7CE52BC0263FFCE5A6
:104E00003F07E1F0A8F0273F3C4539F507E225EEE2
:104E100046EE67EF7CE51DC007E225EE45EE69ED45
:104E20007CE517C006E221EE40EE64EF7CE511C0A0
:104E300007E225EE44EE65EF7CE50BC006E221EECD
:104E400042EE66EF7CE505C008E221E045EE6AED42
:104E50007CE50E94722680E008C0FC0182818823E4
:104E600019F010922B0401C081E00F9108959093E6
:104E700085028093840208959093310480933004D6
:104E80000895E0913004F0913104309721F00190C1
:104E9000F081E02D099480E008950E944127089553
:104EA000E0913004F0913104309721F00280F381D9
:104EB000E02D0994089520912E0430912F04281795
:104EC000390771F090932F0480932E04E091300401
:104ED000F0913104309721F00680F781E02D09949C
:104EE000089520912C0430912D042817390771F072
:104EF00090932D0480932C04E0913004F0913104C0
:104F0000309721F00084F185E02D09940895FC018B
:104F1000329697E080E0915029F021912223D9F335
:104F20008F5FF9CF0895662349F0FC013296089609
:104F30002191621729F0E817F907D1F780E0089569
:104F400081E008959C01FC0132969FEF80E0419141
:104F5000461789F09F3F19F4411101C0982F8F5FC8
:104F60008630A9F79F3F39F0F901E90FF11D97FD50
:104F7000FA956283089508959C012A5F3F4FFC01D2
:104F80004281461301C01282019682179307B9F736
:104F900008950C94A2270C94BC27029626E0FC01ED
:104FA00011922A95E9F7089508950C94D42783E087
:104FB000809332040C94D527811102C081E001C096
:104FC00082E0809332040C94D5270C94DC2781E096
:104FD000809332040C94D5270C94E72708950C9401
:104FE000EE270C94EF270C94EE270C94EE270C94EC
:104FF000EE27CF930E94F5270E9430130E94F327DB
:10500000C0E08C2F0E945A12892B29F4CF5FCA303E
:10501000C1F780E001C081E0CF91089508951F920B
:105020000F920FB60F9211248F939F93AF93BF935C
:1050300080913304811113C08091D3049091D404E2
:10504000A091D504B091D6044196A11DB11D8093C5
:10505000D3049093D404A093D504B093D604BF9105
:10506000AF919F918F910F900FBE0F901F90189549
:105070008091DB04843031F10E94D203109233041A
:1050800020E488E190E00FB6F894A8958093600042
:105090000FBE2093600083B7817F846083BF83B796
:1050A000816083BF7894889583B78E7F83BF0FB666
:1050B000F894A895809160008861809360001092B8
:1050C00060000FBE08950E940F080C94DE0382E07A
:1050D00084BD93E095BD9AEF97BD80936E000895CF
:1050E0002FB7F8948091D3049091D404A091D50463
:1050F000B091D6042FBF08952FB7F8946091D304D0
:105100007091D4048091D5049091D6042FBF089556
:105110009C014FB7F8948091D3049091D404A0914E
:10512000D504B091D6044FBF821B930B0895CF9244
:10513000DF92EF92FF922FB7F894C090D304D090F3
:10514000D404E090D504F090D6042FBFA7019601B7
:10515000261B370B480B590BCA01B901FF90EF9082
:10516000DF90CF90089578941F920F920FB60F9210
:1051700011248F939F93AF93BF938091D304909109
:10518000D404A091D504B091D6040196A11DB11DFF
:105190008093D3049093D404A093D504B093D60401
:1051A000BF91AF919F918F910F900FBE0F901F9065
:1051B000189581E08093E00080E28093D8001092FF
:1051C000C9008FE19EE40197F1F700C0000087E07D
:1051D00090EBDC018093E4049093E504A093E60453
:1051E000B093E7049CE088E10FB6F894A89580930B
:1051F00060000FBE90936000FFCF80913F04089540
:105200000895CF93DF9321E02093E9002FEF3091B1
:10521000E800215035FD06C035ED3A95F1F7000064
:105220002111F5CF2091E80025FF14C0EC0140E0EA
:1052300050E068E070E00E940D2B8091E8008E77CE
:105240008093E80088E0FE01A7E3B4E001900D92AE
:105250008A95E1F7DF91CF9108958093340470939C
:105260003604609335048091DB04843001F582E0DC
:105270008093E9008FEF9091E800815095FD06C082
:1052800095ED9A95F1F700008111F5CF8091E80036
:1052900085FF0DC040E050E063E070E084E394E0FF
:1052A0000E940D2B8091E8008E778093E80008958E
:1052B000BC0184E00C942D29BC0183E00C942D29C1
:1052C00008958091DA04811109C00E949E2C0E94E9
:1052D000FB2C8091E20084608093E200089510929C
:1052E000DA0408950C94EC276091D70481E06111F1
:1052F00001C080E00C94D7279091DB0481E09430CA
:1053000009F080E06091D7040C94DC2742E061EC66
:1053100081E00E94172C42E261EC82E00E94172C8F
:105320009091DB0481E0943009F080E06091D70433
:105330000C94E5278091DD04833009F461C030F4DA
:10534000813071F0823009F49AC008958A3009F4EE
:1053500086C08B3009F46CC0893009F0A8C020C029
:105360008091DC04813A09F0A2C08091E800877F37
:105370008093E8008091E0049091E104892B21F46E
:1053800068E087E394E003C060E080E090E070E0D4
:105390000E94582B8091E8008B778093E800089555
:1053A0008091DC04813209F082C08091E004909108
:1053B000E104029708F07BC08091E800877F80932A
:1053C000E8008091E80082FD05C08091DB04811136
:1053D000F8CF6DC02091F3008091F20090E0922B05
:1053E000029731F48091F100813011F0863021F480
:1053F0008091F10080933F048091E8008B7753C047
:105400008091DC04813A09F052C08091E0049091CF
:10541000E104892B09F04BC08091E800877F8093DD
:10542000E8008091E80080FFFCCF8091E90136C060
:105430008091DC048132D9F58091E0049091E104FF
:10544000892BA9F58091E800877F8093E8000E946E
:105450004C2C8091DE048093E9010C940F0880911C
:10546000DC04813221F58091E800877F8093E80099
:105470000E944C2C8091DF04809340040895809119
:10548000DC04813AA1F48091E800877F8093E800F2
:105490008091E80080FFFCCF809140048093F10070
:1054A0008091E8008E778093E8000C944C2C08954E
:1054B00084B7877F84BF0FB6F894A8958091600069
:1054C000886180936000109260000FBE90E080E8D9
:1054D0000FB6F89480936100909361000FBE0C9416
:1054E000E7270E949E2C0E94FB2CE2EEF0E08081D8
:1054F0008460808378940C94902F8DED91E00C94CF
:105500003C278091DB048530A9F48091DB04853051
:1055100079F40E9438288091D9048823B1F30E943D
:10552000F927882391F30E94F72A0E940F08EDCFF4
:105530000C946328089508950C949E2A292F3327EC
:1055400023303105C9F060F42130310581F022307B
:10555000310509F044C08BE390E022E834E043C019
:1055600021323105E1F02232310549F138C082E1C2
:1055700090E02DEB34E037C099278130910549F058
:1055800028F0029761F5ECE5F4E005C0EEE7F4E001
:1055900002C0EEE6F4E0849190E09F0124C0611522
:1055A000710541F061307105D1F489E090E02DEA98
:1055B00034E019C089E090E024E934E014C06115BA
:1055C000710541F06130710551F482E390E02FECF8
:1055D00034E009C080E490E021E035E004C080E0E0
:1055E00090E020E030E0FA0131832083089580E1EB
:1055F00089BD82E189BD09B400FEFDCF8091D8004C
:105600008F7D8093D8008091E00082608093E000DD
:105610008091E00081FDFCCF0895CF92DF92EF9260
:10562000FF920F931F93CF93DF93EC018B017A01CD
:105630000E946B2C811133C0E114F10439F0F701A1
:1056400080819181081B190BC80FD91FC12CD12C47
:105650000115110519F18091E80085FD16C08091B2
:10566000E8008E778093E800E114F10449F0F70137
:1056700080819181C80ED91ED182C08285E00FC081
:105680000E946B2C882321F30AC089918093F1003A
:1056900001501109FFEFCF1ADF0ADACF80E0DF9166
:1056A000CF911F910F91FF90EF90DF90CF900895D1
:1056B0002091E2043091E3042617370748F0611582
:1056C000710539F42091E8002E772093E80001C09D
:1056D000B901FC0120E06115710579F18091DB04CD
:1056E0008823F1F18530F1F18091E80083FD3CC021
:1056F0008091E80082FD2EC08091E80080FFEBCF12
:105700002091F3008091F20090E0922B61157105D9
:1057100051F08830910538F421912093F1006150C7
:1057200071090196F3CF21E0089709F020E08091FC
:10573000E8008E778093E800CECF2111CFCF0AC04A
:105740008091DB04882361F0853061F08091E8006E
:1057500083FD0AC08091E80082FFF2CF80E00895C7
:1057600082E0089583E0089581E008952091E204A5
:105770003091E3042617370748F06115710539F4B5
:105780002091E8002E772093E80001C0B901FC01C8
:1057900020E06115710591F18091DB04882309F403
:1057A00040C0853009F43FC08091E80083FD3DC0D2
:1057B0008091E80082FD2FC08091E80080FFE9CF52
:1057C0002091F3008091F20090E0922B6115710519
:1057D00059F08830910540F424912093F1003196DE
:1057E000615071090196F2CF21E0089709F020E09D
:1057F0008091E8008E778093E800CBCF2111CCCF49
:105800000AC08091DB04882361F0853061F08091CB
:10581000E80083FD0AC08091E80082FFF2CF80E0BB
:10582000089582E0089583E0089581E00895982F17
:10583000973068F59093E900981739F07091EC0073
:105840002091ED005091F00003C0242F762F50E0FE
:1058500021FD02C09F5FECCF3091EB003E7F309383
:10586000EB003091ED003D7F3093ED003091EB0087
:1058700031603093EB007093EC002093ED00509377
:10588000F0002091EE0027FDE5CF80E008958F70B5
:105890008093E90081E008958091DC0487FF11C0C6
:1058A0008091E80082FD05C08091DB048111F8CF72
:1058B00011C08091E8008B770BC08091DB048823B6
:1058C00049F08091E80080FFF8CF8091E8008E7762
:1058D0008093E80008952091E4003091E50095E67A
:1058E0004091EC00842F817040FF23C08091E8003C
:1058F00080FD1DC08091DB04882399F0853099F0EC
:105900008091EB0085FD11C04091E4005091E500CD
:105910002417350729F3915011F09A01E1CF84E063
:10592000089582E0089583E0089581E0089580E07D
:1059300008954091E80042FFDDCF08950E940C2DAC
:105940000E94142DE0EEF0E0808181608083E8ED1C
:10595000F0E080818F77808319BCA7EDB0E08C9157
:105960008E7F8C9380818F7E80831092DA040895DD
:105970000F931F93CF93DF930E940C2D0E94142D41
:10598000C8EDD0E088818F7788838881806888839C
:1059900088818F7D888319BC1092DB041092D70414
:1059A0001092D9041092D80400EE10E0F801808122
:1059B0008B7F808388818160888342E060E080E023
:1059C0000E94172CE1EEF0E080818E7F8083E2EE72
:1059D000F0E0808181608083808188608083F8012D
:1059E00080818E7F8083888180618883DF91CF91E1
:1059F0001F910F910895E8EDF0E080818F7E808304
:105A0000E7EDF0E080818160808384E082BF81E007
:105A10008093DA040C94B82CE8EDF0E080818E7F5E
:105A200080831092E20008951092DA001092E10053
:105A300008951F920F920FB60F9211242F933F9348
:105A40004F935F936F937F938F939F93AF93BF9386
:105A5000EF93FF938091E10082FF0BC08091E20001
:105A600082FF07C08091E1008B7F8093E1000E945C
:105A70008F2F8091DA0080FF1FC08091D80080FFB7
:105A80001BC08091DA008E7F8093DA008091D9006C
:105A900080FF0DC080E189BD82E189BD09B400FEAF
:105AA000FDCF81E08093DB040E94612905C019BC11
:105AB0001092DB040E946F298091E10080FF19C0E1
:105AC0008091E20080FF15C08091E2008E7F80937C
:105AD000E2008091E20080618093E2008091D80032
:105AE00080628093D80019BC85E08093DB040E941B
:105AF00074298091E10084FF30C08091E20084FF2E
:105B00002CC080E189BD82E189BD09B400FEFDCFD2
:105B10008091D8008F7D8093D8008091E1008F7EA6
:105B20008093E1008091E2008F7E8093E20080917B
:105B3000E20081608093E2008091D704882311F015
:105B400084E007C08091E30087FD02C081E001C0CE
:105B500083E08093DB040E947C298091E10083FF35
:105B600029C08091E20083FF25C08091E100877FFA
:105B70008093E10082E08093DB041092D70480914F
:105B8000E1008E7F8093E1008091E2008E7F809320
:105B9000E2008091E20080618093E20042E060E0F8
:105BA00080E00E94172C8091F00088608093F000C4
:105BB0000E947229FF91EF91BF91AF919F918F91B8
:105BC0007F916F915F914F913F912F910F900FBEF9
:105BD0000F901F9018951F920F920FB60F921124DD
:105BE0002F933F934F935F936F937F938F939F93E5
:105BF000AF93BF93CF93DF93EF93FF93C091E900EF
:105C0000CF708091EC00D82FD17080FDD0E8109239
:105C1000E9008091F000877F8093F00078940E94E3
:105C20002F2E1092E9008091F00088608093F000A0
:105C3000CD2BCF70C093E900FF91EF91DF91CF9111
:105C4000BF91AF919F918F917F916F915F914F9194
:105C50003F912F910F900FBE0F901F9018951F939B
:105C6000CF93DF93CDB7DEB7AA970FB6F894DEBF18
:105C70000FBECDBFECEDF4E08091F100819324E004
:105C8000E43EF207C9F70E949A298091E80083FF59
:105C90002EC18091DC049091DD04492F50E04A3000
:105CA000510508F024C1FA01E857FF4F0C94053064
:105CB000803821F0823809F01AC108C08091D804D8
:105CC0009091D904992389F082600FC08091E004FB
:105CD0008F70873008F00BC18093E9008091EB0052
:105CE00085FB882780F91092E9009091E800977F62
:105CF0009093E8008093F1001092F100D1C0282F1A
:105D00002D7F09F0F4C0882319F0823061F0EFC0D4
:105D10008091DE04813009F0EAC0933009F080E020
:105D20008093D9042EC08091DE0481112AC0809115
:105D3000E0048F702FEF280F263008F0D8C0809332
:105D4000E9002091EB0020FF1CC0933021F48091EA
:105D5000EB00806214C09091EB0090619093EB0097
:105D600021E030E0A90102C0440F551F8A95E2F7F7
:105D70004093EA001092EA008091EB0088608093E3
:105D8000EB001092E9008091E800877F8093E800A3
:105D90000E944C2CACC08111AAC01091DE041F7768
:105DA0008091E3008078812B8093E3008091E8006C
:105DB000877F8093E8000E944C2C8091E80080FF50
:105DC000FCCF8091E30080688093E300111102C052
:105DD00082E001C083E08093DB0489C08058823078
:105DE00008F085C08091DE049091DF048C3D53E083
:105DF000950779F583E08A838AE289834FB7F8941F
:105E0000DE01139620E03EE051E2E32FF0E05093F4
:105E10005700E49120FF03C0E295EF703F5FEF7001
:105E20008E2F90E0EA3010F0C79601C0C0968D9397
:105E30009D932F5F243149F74FBF8091E800877F02
:105E40008093E8006AE270E0CE0101960E94582B30
:105E500016C06091E0047091E104AE014F5F5F4FA6
:105E60000E949C2ABC01892B09F441C09091E80052
:105E7000977F9093E80089819A810E94B62B809148
:105E8000E8008B778093E80032C0803881F58091FC
:105E9000E800877F8093E8008091D7048093F10029
:105EA0008091E8008E7772CF811121C08091DE044D
:105EB0009091DF0499270297D4F48091E800877FBE
:105EC0008093E8008091DE048093D7040E944C2CDC
:105ED0008091D704811106C08091E30087FD02C044
:105EE00081E001C084E08093DB040E9486298091D8
:105EF000E80083FF0AC08091E800877F8093E80074
:105F00008091EB0080628093EB00AA960FB6F89424
:105F1000DEBF0FBECDBFDF91CF911F9108950895D1
:105F2000CF938091DB048823A1F0C091E900CF706A
:105F30009091EC00892F817090FD80E8C82B109221
:105F4000E9008091E80083FD0E942F2ECF70C0935E
:105F5000E900CF910895DB018F939F930E941A303F
:105F6000BF91AF91A29F800D911DA39F900DB29FF5
:105F7000900D11240895AA1BBB1B51E107C0AA1F55
:105F8000BB1FA617B70710F0A61BB70B881F991FDA
:105F90005A95A9F780959095BC01CD01089597FB7E
:105FA000072E16F4009407D077FD09D00E94BB2F6E
:105FB00007FC05D03EF4909581959F4F089570950C
:105FC00061957F4F0895A1E21A2EAA1BBB1BFD010C
:105FD0000DC0AA1FBB1FEE1FFF1FA217B307E407C8
:105FE000F50720F0A21BB30BE40BF50B661F771F20
:105FF000881F991F1A9469F7609570958095909500
:106000009B01AC01BD01CF010895EE0FFF1F05906C
:10601000F491E02D0994A29FB001B39FC001A39F0A
:10602000700D811D1124911DB29F700D811D1124D1
:10603000911D08950E940B30A59F900DB49F900D67
:10604000A49F800D911D112408958F929F92AF926D
:10605000BF92CF92DF92EF92FF92CF93DF93EC014A
:10606000688179818A819B8161157105810591051E
:1060700021F464E279ED8BE597E02DE133EF41E027
:1060800050E00E94E03049015A019B01AC01A7EAAF
:10609000B1E40E941A306B017C01ACEEB4EFA501B3
:1060A00094010E940231DC01CB018C0D9D1DAE1DBF
:1060B000BF1DB7FF03C00197A109B048888399832A
:1060C000AA83BB839F77DF91CF91FF90EF90DF9002
:1060D000CF90BF90AF909F908F9008950E942530F1
:1060E000089580E091E00E9425300895A0E0B0E09E
:1060F0008093000190930101A0930201B0930301EA
:106100000895FB01DC0104C08D910190801921F4F8
:1061100041505040C8F7881B990B0895DC01CB0112
:10612000FC01F999FECF06C0F2BDE1BDF89A3196A7
:1061300000B40D9241505040B8F70895F999FECF40
:1061400092BD81BDF89A992780B50895A8E1B0E085
:1061500042E050E00C949030DC01A40FB51F415098
:10616000504048F0CB01840F951F2E910E94BD3006
:1061700041505040D0F70895262FF999FECF92BD97
:1061800081BDF89A019700B4021639F01FBA20BDFC
:106190000FB6F894FA9AF99A0FBE08950396272F2E
:1061A0000E94BD300E94BC30252F0E94BD30242F9C
:1061B0000C94BD300196272F0E94BD300C94BC304A
:1061C000052E97FB1EF400940E94F73057FD07D070
:1061D0000E94E32F07FC03D04EF40C94F730509547
:1061E0004095309521953F4F4F4F5F4F08959095C3
:1061F0008095709561957F4F8F4F9F4F0895B7FFA2
:106200000C941A300E941A30821B930B0895F89454
:02621000FFCFBE
:1062120001000000121110FF0F0EFFFF0D0CFFFF17
:10622200FFFFFFFFFFFFFFFFFFFF13FFFFFFFFFF68
:10623200FFFFFFFFFFFFFFFFFFFFFFFFFFFFFFFF6C
:1062420014FFFFFFFF18FFFF1AFFFF151617191B98
:10625200FF1C1DFF00010B0AFF09FF08FF0706FFD5
:1062620005FFFFFFFFFFFFFFFFFFFF04FFFFFFFF31
:10627200FFFFFFFFFFFF03FFFFFFFFFFFFFFFFFF28
:10628200FF0200001200250038004A005D00700085
:1062920082009500A800BA00CD000019CD19003384
:1062A200CD33003F123F253F383F4A3F5D3F703FAD
:1062B200823F953FA83FBA3FCD3F0000000000005B
:1062C20001010101010101010101010101010101BC
:1062D200010101010101010101010101010100C8E6
:1062E2000018030300FF00FFFF39050601FD280126
:1062F2002960295C29582900290100FFFFE200E9F1
:1063020000EA00B500B600B700CD008301CC008AD8
:10631200019201940121022302240225022602276E
:10632200022A02B300B4006F007000818283E2008F
:10633200E900EA00B500B600B700CD008301CC0049
:106342008A019201940121022302240225022602DB
:1063520027022A02B300B4006F007000818283F02A
:10636200C6309091929395949697F7F6F5F4F1676B
:1063720034353666003131295A1B750AF220F32072
:10638200FF200B2100FF0100010000FFFF000001C0
:046392000001FF0007
:00000001FF
